:10000000B2019029A501A400B3172730A300103036
:1000100015200330A300E8301520A301643015201B
:10002000A3010A30152024082028A2002508A100D9
:100030002408A00069212008031DB313B31B080086
:10004000303EA7008611051205128316861105128F
:100050000512F030850583122708B2184D283A3072
:10006000A10098303E213330A60062201330A10059
:1000700088303E21622064303D21622064303D2181
:100080002230A600622028304C200C304C20063054
:100090004C20B21427084D283214A600321C5B28CD
:1000A0000512033C031C602860200730A100D030FB
:1000B0003E21031408003214FE3C03198B29051657
:1000C000A60E321C32108615F030850526080F3931
:1000D00085048611A60E3218622832303D210314A1
:1000E0000800B4002C212008210403198B29852144
:1000F00084133408800664007D287E28A00A031932
:10010000A10F7B2880068B293708A0003508A100A5
:100110000130A200A3016400AC20031C9F28A20BA5
:100120008B28FF30A30703188B28A007031CA10707
:10013000031C8B293230A2000030A3008B28DD2065
:100140000830A300DE20AC20A20CA628A30BA22816
:10015000DE200314220808003608840034088417BF
:1001600080048413000533193406FF3E0800A600FE
:10017000360884000930A7000310C320A60CA70B83
:10018000BD280314C3288413B31DD22800083404E7
:10019000331D34068000841700083404031C340621
:1001A0008000DE2800083404031C340633193406AA
:1001B0008000841734098005DE283317330D063993
:1001C000A000EC20A100A00AEC20331F3E2933132D
:1001D000A000023064213E2900308A0020088207F6
:1001E000013475340334153400343C340C34D934C0
:1001F0000830A600A70037088400350833192421E9
:10020000331D26213608840034082921A001A101CC
:10021000260803198B29B3181D213608840000080D
:100220003405FF3EA00DA10DB31C1D21A60B0B290B
:1002300027083318522920088B29370884003508ED
:10024000800600008006080080042C29FF3A800503
:100250002D29841780048B29FF3A841780058B2968
:10026000A301A200FF30A207031CA307031C8B29D4
:100270000330A100DF303E213229A101E83EA00079
:10028000A109FC30031C4729A00703184429A00733
:100290006400A10F442920184D29A01C51290000F9
:1002A00051290800A201A3015929A10CA00CA20DFB
:1002B000A30DFF3E031855292308A1002208A00022
:1002C0008B290310A10CA00CFF3E03186129200804
:1002D0008B29A501A4011030A600210DA40DA50DA8
:1002E0002208A4022308031C230FA50203187F2958
:1002F0002208A40723080318230FA5070310A00D45
:10030000A10DA60B6D2920088B29A009A109A00A1F
:100310000319A10A08008313031383126400080061
:1003200007309F0006138316061383120130B900AD
:10033000C8303021FE302120013021200130A300BF
:10034000F4303121FE302120023021204C30212098
:1003500043302120443021202030212072302120C0
:100360006530212061302120643021207930212026
:100370000130A300F4303121FE3021200130212052
:10038000FE302120023021205430212065302120F0
:100390007330212074302120203021204230212050
:1003A0006F302120613021207230212064302120E3
:1003B000203021203A080220FE302120C0302120A8
:1003C000533021206530212072302120203021201F
:1003D00044302120613021207430212061302120DF
:1003E00020302120493021206E3021202030212052
:1003F000380802200630B6008030B4000430B30064
:100400009B30B700B5018420031C092AB8000530D1
:1004100030210630B6004030B4000430B3003A0852
:10042000B7200130A000A101063084000130712006
:1004300006128316061205308312B6004030B4004F
:100440000630B7002030B500B301F820BA00061618
:1004500083160612640083123A083B020319322AFB
:100460000130B90064003A083B02031D3F2AB90A73
:10047000640010303902031C3F2A0130B9006400C7
:0E048000023039020318C0293A08BB00C02917
:02400E00543F1D
:00000001FF
